:1000000010C02AC029C028C027C026C025C024C0CF
:1000100023C022C021C020C01FC01EC01DC01CC0E4
:100020001BC011241FBECFE5D1E0DEBFCDBF10E065
:10003000A0E6B0E0E2EFF2E002C005900D92A23837
:10004000B107D9F720E0A2E8B0E001C01D92A03AC4
:10005000B207E1F70ED14BC1D3CFFC01DA011C92FC
:1000600090819623E9F78CE18A95F1F7000088E307
:100070008A95F1F700C08081862319F08C91816008
:100080008C9388E38A95F1F700C08081862319F06C
:100090008C9182608C9388E38A95F1F700C080810F
:1000A000862319F08C9184608C9388E38A95F1F70C
:1000B00000C08081862319F08C9188608C9388E33E
:1000C0008A95F1F700C08081862319F08C918061B8
:1000D0008C9388E38A95F1F700C08081862319F01C
:1000E0008C9180628C9388E38A95F1F700C08081BF
:1000F000862319F08C9180648C9388E38A95F1F7BC
:1001000000C08081682319F08C9180688C9388E30B
:100110008A95F1F700C08CE18A95F1F70000089507
:10012000FC019081862F80959823908398E39A957F
:10013000F1F700C040FF04C09081962B908303C06C
:1001400090819823908398E39A95F1F700C041FF3E
:1001500004C09081962B908303C090819823908354
:1001600098E39A95F1F700C042FF04C09081962B66
:10017000908303C090819823908398E39A95F1F738
:1001800000C043FF04C09081962B908303C09081F0
:100190009823908398E39A95F1F700C044FF04C038
:1001A0009081962B908303C090819823908398E34D
:1001B0009A95F1F700C045FF04C09081962B90837B
:1001C00003C090819823908398E39A95F1F700C03B
:1001D00046FF04C09081962B908303C090819823A2
:1001E000908398E39A95F1F700C0442324F480812A
:1001F000862B808303C090818923808388E38A953E
:10020000F1F700C08081682B608398E39A95F1F73D
:1002100000C088E38A95F1F700C00895FF920F931C
:100220001F93CF93DF93EC01F62E8A0110929F006B
:1002300010929E00E0919E00F0919F00E00FF11F50
:1002400040816F2DCE016CDF80919E0090919F00C8
:10025000019690939F0080939E00F801E80FF91F8C
:1002600080818111E7CFDF91CF911F910F91FF9096
:10027000089580E886BD16BCD99AD19A10929D0047
:1002800010929C004BE950E061E089E390E0E5DEEC
:1002900040E650E062E08BE390E0C0DF80919C009C
:1002A00090919D009C012F5F3F4F30939D002093C4
:1002B0009C00FC01EE57FF4F40919B00408328318A
:1002C000310521F410929D0010929C0042E850E00C
:1002D00062E08BE390E0A2DF42E262E08BE390E039
:1002E0001FDF4AE062E08BE390E01ADFCBCFF894A7
:0202F000FFCF3E
:1002F20068656C6C6F2E667464692E34342E656387
:10030200686F2E633A20796F752074797065642066
:020312002200C7
:00000001FF
